:020000020000FC
:0200000007C037
:10000E0014C01FED1DBF789410E215BFA3D1ABD164
:10001E006EEA78E510E185ED93E861D110E1862F67
:10002E00972F5DD133278895FECF0FB61AB11F7764
:10003E001AB95F9BFECF4CB13395313091F032300F
:10004E0099F03330A1F03430A9F03530B1F03630BC
:10005E00B9F03730C1F03830C9F03930C9F03A3024
:10006E00C9F024D085D118952AD082D1189530D0D8
:10007E007FD1189540D07CD118957AD079D118952A
:10008E00B4D076D11895EED073D1189571D118954C
:10009E006FD1189572D110E185ED93E820D110E162
:1000AE00862F972F1CD1332763D11895142F4033E9
:1000BE0019F033275DD1189560E070E00895142F84
:1000CE00403319F0332754D1189560E070E008954D
:1000DE00142F403339F0413341F0423349F0332786
:1000EE0047D1189560E070E0089560E177E20895D9
:1000FE0060E27EE40895142F4033A9F04133A1F05D
:10010E004233B1F04333C1F04433D1F04533E1F023
:10011E004633F1F0473301F1483311F1493321F100
:10012E00332726D11895089588EE93E019D10895B6
:10013E0080ED97E015D1089588EB9BE011D10895DD
:10014E0080EA9FE00DD1089588E893E109D10895E2
:10015E0080E797E105D1089588E59BE101D10895E7
:10016E0080E49FE1FDD0089588E293E2F9D00895EE
:10017E00142F4033A9F04133A1F04233B1F0433391
:10018E00C1F04433D1F04533E1F04633F1F047335B
:10019E0001F1483311F1493321F13327E9D0189594
:1001AE00089584E690E0DCD0089588EC90E0D8D0F5
:1001BE0008958CE291E0D4D0089580E991E0D0D0FA
:1001CE00089584EF91E0CCD0089588E592E0C8D0F0
:1001DE0008958CEB92E0C4D0089580E293E0C0D0F5
:1001EE00089584E893E0BCD00895142F4033A9F00D
:1001FE004133A1F04233B1F04333C1F04433D1F077
:10020E004533E1F04633F1F0473301F1483311F154
:10021E00493321F13327ACD0189508958AE090E048
:10022E009FD0089584E190E09BD008958EE190E0F8
:10023E0097D0089588E290E093D0089582E390E0FD
:10024E008FD008958CE390E08BD0089586E490E0F3
:10025E0087D0089580E590E083D008958AE590E0F8
:10026E007FD00895142F4033A9F04133A1F04233CB
:10027E00B1F04333C1F04433D1F04533E1F04633AE
:10028E00F1F0473301F1483311F1493321F13327AE
:10029E006FD01895089581E090E062D0089582E0C5
:1002AE0090E05ED0089583E090E05AD0089584E007
:1002BE0090E056D0089585E090E052D0089586E003
:1002CE0090E04ED0089587E090E04AD0089588E0FF
:1002DE0090E046D0089589E090E042D00895C3980A
:1002EE0022E02A95F1F7C498C39A27E02A95F1F7F0
:1002FE00C29A27E02A95F1F7C2980000880F991F3D
:10030E0010F0C49807C022E02A95F1F7C49A23E0B2
:10031E002A95F1F722E02A95F1F7C29A27E02A955D
:10032E00F1F7C2981A9549F722E02A95F1F70000E5
:10033E00C49AC3980000000000000000C29A00009A
:10034E00000000000000C29827E02A95F1F7C29A3B
:10035E00C39A08951FEF17BBC29AC39AC49A089501
:10036E00680F791F08951CE019B918E91AB9089594
:10037E001AB110681AB90FBE08958EEC99E2680F83
:04038E00791F089536
:00000001FF
